:100000000C9437010C9454010C9454010C94540139
:100010000C9454010C9454010C9454010C9454010C
:100020000C9454010C9454010C9454010C945401FC
:100030000C94D1120C9454010C9454010C9454015E
:100040000C9454010C94B5050C9407190C94E6110A
:100050000C9470120C9454010C9454010C9454019F
:100060000C9454010C9454010C9454010C945401BC
:100070004570692D4F5344205665722E302E392E0F
:10008000312E380000416B7475656C6C65732053BC
:10009000657474696E67000053657474696E6720D7
:1000A000200000486F6568656E73656E736F72201F
:1000B00000004853206D697420536368616C746557
:1000C0007220000048656164696E6720486F6C6447
:1000D0002000004B6F6D706173732000004B6F6DDB
:1000E0007061737320666978200000475053204187
:1000F0006B74697620000041636873656E6B6F7086
:1001000070656C756E67200000447265687261747A
:100110006520626567722E2000004665686C657216
:100120002046433C2D3E4F5344200000556E7465DD
:10013000727370616E6E756E672000004B65696E3C
:10014000652053657474696E672D416E7A656967C1
:1001500065000050432F425420616B7469760000A3
:1001600055656265726E65686D65204C65747A745C
:1001700065732053657474696E6700004B65696E22
:1001800065204465766976652D416E7A6569676597
:10019000000050432F425420616B74697600005573
:1001A000656265726E65686D65204C65747A74650C
:1001B000732044657669636500004F4E00002D2D65
:1001C0002D000044657669636520756E6420566570
:1001D0007273696F6E736162667261676500004475
:1001E000656369766520202020203D200000465769
:1001F0002D56657273696F6E203D200000464300E6
:10020000004E43000046432D6F6C642046570000AB
:100210004550492D4D656E750050616C0050432F5F
:100220004254004B656E6E756E670052432D4265F9
:100230007472696562004550492D5374726F6D0088
:1002400045786974004F4E002D2D0076767D7676C8
:100250007A76767E76767776767B76767876767C24
:1002600076767976767D76767A76767E7600112445
:100270001FBECFEFD4E0DEBFCDBF11E0A0E0B1E004
:10028000E2E2F4E302C005900D92A039B107D9F77C
:1002900013E0A0E9B1E001C01D92A43BB107E1F772
:1002A0000E9464010C940F1A0C94000086E981BB33
:1002B0008FE084BBAC9AAD9A8EE28ABB80EB87BBA1
:1002C000C69AD99ADD9A08951092D8011092D40155
:1002D0001092D901E199FECF80E090E09FBB8EBBE8
:1002E000E09A8DB380939701E199FECF81E090E091
:1002F0009FBB8EBBE09A8DB380930001E199FECF46
:1003000082E090E09FBB8EBBE09A8DB38093980112
:10031000E199FECF87E190E09FBB8EBBE09A8DB361
:100320008093A501E199FECF88E190E09FBB8EBB51
:10033000E09A8DB38093BE01E199FECF8AE190E00F
:100340009FBB8EBBE09A8DB380930901E199FECFEC
:1003500089E190E09FBB8EBBE09A8DB38093BA0198
:10036000E199FECF8BE190E09FBB8EBBE09A8DB30D
:100370008093990120910001213079F49EE09093BF
:10038000030187E08093040186E8809305012093B0
:100390000601909307018CE00EC09CE0909303014E
:1003A00085E0809304018AE48093050110920601A0
:1003B000909307018AE0809308010E942F170E9402
:1003C00056010E94AE0580919701813019F40E9478
:1003D000C11002C00E94B1107894A89A0E94E4044F
:1003E0000E9416060E94090A80919901882311F043
:1003F0000E94490A8091C301882311F00E949F1333
:100400000E94490A80919901813011F40E94571984
:100410000E9492118091B601813021F41092B601B0
:100420000E94C7178091DD01813021F41092DD0117
:100430000E94DF0D809192018130E9F410929201C7
:100440008091D801882389F48091BA01843069F4BD
:1004500080919701882349F480919A01813029F491
:1004600080E363E64AE00E9440110E94C4120E94A9
:10047000C9120E94721480919901813031F48091E7
:10048000DE01813011F40E94621980919501813062
:10049000E1F48091D8018823C1F4AA9A0E94060F42
:1004A0000E9469090E947E088091C101882321F081
:1004B0000E943D130E94C70A8091C201882311F057
:1004C0000E9477170E949E0AAA988091900181301D
:1004D00069F58091D801882349F5109290018091A7
:1004E000A501882321F080910201833014F00E943D
:1004F000780A8091A2019091A30101969093A301A3
:100500008093A2010197CB9769F48091A00190910B
:10051000A10101969093A1018093A0011092A301E3
:100520001092A2010E94570C0E94A10D809191018E
:10053000813009F06FCF8091D801882309F06ACF0C
:100540001092910180919901813039F48091DE01FE
:10055000882319F481E00E9462190E94120A809196
:10056000C301882309F456CF0E94F7130E94D013C9
:100570000E94A7134FCF782FD99827E030E041E0B1
:1005800050E0DB980000000000000000CA01022ECD
:1005900002C0880F991F0A94E2F7872311F0DA9AB4
:1005A00001C0DA980000000000000000DB9A0000A3
:1005B000000000000000215030408FEF2F3F38072F
:1005C00001F727E030E041E050E0DB980000000058
:1005D00000000000CA01022E02C0880F991F0A9471
:1005E000E2F7862311F0DA9A01C0DA9800000000E1
:1005F00000000000DB9A0000000000000000215015
:1006000030408FEF2F3F380701F7DB98DA98D99AFF
:10061000089584E064E00E94BB0280E06CE40E94E4
:10062000BB0210929201809192018823E1F38CE643
:100630006AE00E94BB0285E060E00E94BB02089570
:100640001F938091BA01823051F40E94D110109210
:100650009001809190018823E1F31092900182E64D
:1006600061E74FEF0E9440111092900110E00DC021
:1006700080919501813011F40E94060F80919001C4
:10068000813019F41092900111E08091C00188230B
:1006900011F4112369F38091BA01823011F40E94A0
:1006A0001811112309F0D9C08091A3038093090187
:1006B000809193038093BE012091BE01E199FECF0A
:1006C00088E190E09FBB8EBB2DBB0FB6F894E29AF9
:1006D000E19A0FBE20910901E199FECF8AE190E0F5
:1006E0009FBB8EBB2DBB0FB6F894E29AE19A0FBE6A
:1006F00082E061E045E850E00E94410E82E062E065
:1007000048E950E00E94410E82E064E043EA50E094
:100710000E94410E82E065E042EB50E00E94410EF3
:1007200082E066E044EC50E00E94410E82E067E027
:1007300043ED50E00E94410E82E068E04DED50E054
:100740000E94410E82E069E04BEE50E00E94410EB3
:1007500082E06AE047EF50E00E94410E82E06BE0E9
:100760004CE251E00E94410E4091BC015091BD010C
:1007700084E162E00E94B40D8091BE0180FF05C05B
:1007800084E164E04AEB51E004C084E164E04EEBB4
:1007900051E00E94410E8091BE0181FF05C084E1BD
:1007A00065E04AEB51E004C084E165E04EEB51E0C6
:1007B0000E94410E8091BE0182FF05C084E166E087
:1007C0004AEB51E004C084E166E04EEB51E00E9448
:1007D000410E8091BE0183FF05C084E167E04AEBD2
:1007E00051E004C084E167E04EEB51E00E94410E0D
:1007F0008091BE0184FF05C084E168E04AEB51E0CE
:1008000004C084E168E04EEB51E00E94410E80910B
:10081000BE0185FF05C084E169E04AEB51E004C0F8
:1008200084E169E04EEB51E00E94410E8091BE01EF
:1008300086FF05C084E16AE04AEB51E004C084E130
:100840006AE04EEB51E00E94410E4091090184E1C3
:100850006BE050E00E94B40D20C082E062E045E809
:1008600050E00E94410E82E065E04AE151E00E94C2
:10087000410EE199FECF88E190E09FBB8EBBE09AEC
:100880008DB380939303E199FECF8AE190E09FBB03
:100890008EBBE09A8DB38093090190919303892FC9
:1008A00081708093C101892F88708093C201892F44
:1008B00080728093C30194709093C4011F91089536
:1008C0001F93809190018823E1F31092900183E6B9
:1008D00066E740E00E94401110E00DC08091950154
:1008E000813011F40E94E90E80919001813019F459
:1008F0001092900111E08091BB01882311F4112323
:1009000069F3112309F054C082E062E043EC51E046
:100910000E94410E82E064E04FED51E00E94410EE2
:1009200082E066E04EEE51E00E94410E8091BA01F5
:10093000813031F48EE064E04DEF51E00E94410ED1
:100940008091BA01823031F48EE064E041E052E0FF
:100950000E94410E8091BA01843031F48EE064E04F
:1009600045E052E00E94410E40914D038EE066E06A
:1009700050E00E94B40D40914E0380E166E050E0EB
:100980000E94B40D40914F0383E166E050E00E9465
:10099000B40D2091BA01E199FECF89E190E09FBBAF
:1009A0008EBB2DBB0FB6F894E29AE19A0FBE0AC037
:1009B000E199FECF89E190E09FBB8EBBE09A8DB3B9
:1009C0008093BA011F9108950E94090383E66FE6A0
:1009D00044E60E944011109290018091900188237A
:1009E000E1F387E062E040E750E00E94410E0E94A0
:1009F000170610929001809190018823E1F31092E4
:100A00009001809190018823E1F3109290018091F0
:100A100090018823E1F31092900184E064E00E9449
:100A2000BB0280E06CE40E94BB02809197018823A6
:100A300019F40E9460041CC082E062E04CE751E0BF
:100A40000E94410E82E064E042E951E00E94410EC2
:100A500082E066E04FE951E00E94410EE199FECF4D
:100A600089E190E09FBB8EBBE09A8DB38093BA0181
:100A7000809190018823E1F3109290018091900180
:100A80008823E1F31092900184E064E00E94BB02AD
:100A900080E06CE40E94BB0280919701882319F4E6
:100AA0000E94200326C082E062E04CE351E00E94F5
:100AB000410E82E064E043E551E00E94410E82E095
:100AC00066E040E651E00E94410EE199FECF88E1E8
:100AD00090E09FBB8EBBE09A8DB38093BE01E199FD
:100AE000FECF8AE190E09FBB8EBBE09A8DB38093EE
:100AF00009018091BA01823029F483E66FE64AE069
:100B00000E9440118091BA01813029F482E664E6A6
:100B10004AE00E944011809190018823E1F31092F5
:100B20009001809190018823E1F3109290018091CF
:100B300090018823E1F31092900180919001882325
:100B4000E1F310929001809190018823E1F31092DB
:100B5000900184E064E00E94BB02089582E083BFBC
:100B600082E48EBD8AE089BF08951F920F920FB66E
:100B70000F9211248F939F93809194018F5F8093A4
:100B8000940180919401883449F591E09093930108
:100B9000109294018091AA038F5F8093AA038091A1
:100BA000AA03843631F41092AA0390939001909393
:100BB00091018091AA03823319F481E0809391011D
:100BC0008091A9038F5F8093A9038091A9038A3044
:100BD00029F41092A90381E0809392019F918F9153
:100BE0000F900FBE0F901F901895982F80538A304A
:100BF00010F020E005C0903311F42AE001C0282F46
:100C0000892F81548A3110F4292F2653892F815638
:100C10008A3110F4292F2C539D3211F429E403C09A
:100C20009E3209F421E4822F08950895089585E005
:100C300060E00E94BB0286E063E80E94BB0287E09E
:100C400060E90E94BB0285E060E00E94BB0286E092
:100C500064E80E94BB0287E061E90E94BB0285E074
:100C600060E00E94BB0286E065E80E94BB0287E06C
:100C700062E90E94BB0285E060E00E94BB0286E060
:100C800066E80E94BB0287E063E90E94BB0285E040
:100C900060E00E94BB0286E067E80E94BB0287E03A
:100CA00064E90E94BB0285E060E00E94BB0286E02E
:100CB00068E80E94BB0287E065E90E94BB0285E00C
:100CC00060E00E94BB0286E069E80E94BB0287E008
:100CD00066E90E94BB0285E060E00E94BB0286E0FC
:100CE0006AE80E94BB0287E067E90E94BB0285E0D8
:100CF00060E00E94BB0286E061EA0E94BB0287E0DE
:100D000068E90E94BB0285E060E00E94BB0286E0C9
:100D100062EA0E94BB0287E069E90E94BB0285E0AB
:100D200060E00E94BB0286E063EA0E94BB0287E0AB
:100D30006AE90E94BB0285E060E00E94BB0286E097
:100D400064EA0E94BB0287E06BE90E94BB0285E077
:100D500060E00E94BB0286E065EA0E94BB0287E079
:100D60006CE90E94BB0285E060E00E94BB0286E065
:100D700066EA0E94BB0287E06DE90E94BB0285E043
:100D800060E00E94BB0286E067EA0E94BB0287E047
:100D90006EE90E94BB0285E060E00E94BB0286E033
:100DA00068EA0E94BB0287E06FE90E94BB0285E00F
:100DB00060E00E94BB0286E06FEB0E94BB0287E00E
:100DC00060EA0E94BB0285E060E00E94BB0286E010
:100DD00060EC0E94BB0287E061EA0E94BB0285E0F2
:100DE00060E00E94BB0286E061EC0E94BB0287E0EB
:100DF00062EA0E94BB0285E060E00E94BB0286E0DE
:100E000062EC0E94BB0287E063EA0E94BB0285E0BD
:100E100060E00E94BB0286E063EC0E94BB0287E0B8
:100E200064EA0E94BB0285E060E00E94BB0286E0AB
:100E300064EC0E94BB0287E065EA0E94BB0285E089
:100E400060E00E94BB0286E065EC0E94BB0287E086
:100E500066EA0E94BB0285E060E00E94BB0286E079
:100E600066EC0E94BB0287E067EA0E94BB0285E055
:100E700060E00E94BB0286E06DED0E94BB0287E04D
:100E800068EA0E94BB0285E060E00E94BB0286E047
:100E90006EED0E94BB0287E069EA0E94BB0285E01A
:100EA00060E00E94BB0286E06FED0E94BB0287E01B
:100EB0006AEA0E94BB0285E060E00E94BB0286E015
:100EC00060EE0E94BB0287E06BEA0E94BB0285E0F5
:100ED00060E00E94BB0286E061EE0E94BB0287E0F8
:100EE0006CEA0E94BB0285E060E00E94BB0286E0E3
:100EF00062EE0E94BB0287E06DEA0E94BB0285E0C1
:100F000060E00E94BB0286E063EE0E94BB0287E0C5
:100F10006EEA0E94BB0285E060E00E94BB0286E0B0
:100F200064EE0E94BB0287E06FEA0E94BB0285E08C
:100F300060E00E94BB0286E06BEF0E94BB0287E08C
:100F400060EB0E94BB0285E060E00E94BB0286E08D
:100F50006CEF0E94BB0287E061EB0E94BB0285E060
:100F600060E00E94BB0286E06DEF0E94BB0287E05A
:100F700062EB0E94BB0285E060E00E94BB0286E05B
:100F80006EEF0E94BB0287E063EB0E94BB0285E02C
:100F900060E00E94BB0286E06FEF0E94BB0287E028
:100FA00064EB0E94BB0285E061E00E94BB0286E028
:100FB00060E00E94BB0287E065EB0E94BB0285E017
:100FC00061E00E94BB0286E061E00E94BB0287E014
:100FD00066EB0E94BB020895BF92CF92DF92EF9220
:100FE000FF920F931F93CF93DF937C01B62E8C015A
:100FF00045E0C42ED12CC80ED91E862F90E0EC01FE
:10100000CC0FDD1FC80FD91FCA5EDE4F0EC085E0B2
:10101000612F0E94BB0286E0602F0E94BB0287E026
:1010200068810E94BB020F5F1F4F0C151D0578F3EE
:101030008701065F1F4F8FE090E0E80EF91E8B2DB1
:1010400090E0EC01CC0FDD1FC80FD91FCA5EDE4F48
:101050000EC085E0612F0E94BB0286E0602F0E94D7
:10106000BB0287E068810E94BB020F5F1F4F0E1515
:101070001F0578F3DF91CF911F910F91FF90EF90B3
:10108000DF90CF90BF900895EF92FF920F931F9340
:10109000CF93DF938C01EC0155E0E52EF12CE80EA7
:1010A000F91E0DC085E06D2F0E94BB0286E06C2FFB
:1010B0000E94BB0287E060E00E94BB022196CE1531
:1010C000DF0580F3E8012A96015F1F4F0DC085E020
:1010D0006D2F0E94BB0286E06C2F0E94BB0287E04E
:1010E00060E00E94BB022196C017D10780F3DF9118
:1010F000CF911F910F91FF90EF9008951F93CF9381
:10110000DF93C0914D02D0914E02D7FD12C0CE01A7
:101110006AE070E00E94FC19182F169520910401D6
:1011200030E0CE016AE070E00E94FC19261B310914
:1011300018C0EE27FF27EC1BFD0BCF016AE070E023
:101140000E94FC19182F16951C5F2091040130E0B5
:101150002F5F3F4FCF016AE070E00E94FC19260F1D
:10116000311DE90175E0CC0FDD1F7A95E1F7220F03
:10117000331FC21BD30B279680911201909113014C
:10118000C817D90739F080911201909113010E947C
:10119000440804C08091C701811721F0CE01612F5E
:1011A0000E94EC071093C701D0931301C093120162
:1011B000DF91CF911F910895CF92DF92EF92FF922E
:1011C0000F931F93CF93DF938C01E62E85E0612F61
:1011D0000E94BB0286E0602F0E94BB02CE2CDD2461
:1011E00084E391E0C80ED91E87E0F60160810E9479
:1011F000BB02EEE1EE2EF12CE00EF11E85E06F2D2C
:101200000E94BB0286E06E2D0E94BB0287E0F601C1
:1012100060810E94BB02E801CC54DF4F025F1E4F89
:1012200085E06D2F0E94BB0286E06C2F0E94BB02FE
:1012300087E0F60160810E94BB026E96C017D1075D
:1012400079F7DF91CF911F910F91FF90EF90DF9091
:10125000CF900895EF92FF920F931F93CF93DF9358
:101260007C0185E06F2D0E94BB0286E06E2D0E94FE
:10127000BB0287E060E00E94BB028701025E1F4F55
:1012800085E0612F0E94BB0286E0602F0E94BB02B6
:1012900087E060E00E94BB02E701CC54DF4F87018A
:1012A000025F1E4F85E06D2F0E94BB0286E06C2F0F
:1012B0000E94BB0287E060E00E94BB026E96C017EE
:1012C000D10781F7DF91CF911F910F91FF90EF90A0
:1012D00008951F93CF93DF93E0914B02F0914C025E
:1012E000F7FD14C0CF016AE070E00E94FC19182FCE
:1012F00016951C5F80910501C82FD0E0CF016AE0F0
:1013000070E00E94FC19C61BD10917C022273327A1
:101310002E1B3F0BC9016AE070E00E94FC19182FD8
:10132000169580910501C82FD0E02196C9016AE089
:1013300070E00E94FC19C60FD11D8091140190919C
:101340001501C817D90739F0809114019091150142
:101350000E942A0904C08091C801811721F0CE01A2
:10136000612F0E94DC081093C801D0931501C0932F
:101370001401DF91CF911F91089585E060E00E94F4
:10138000BB0286E06FEC0E94BB0287E06CE80E9423
:10139000BB0285E061E00E94BB0286E06BE00E9438
:1013A000BB0287E06DE80E94BB020895EF92FF92B6
:1013B0000F931F93CF93DF937A019EE1699FB00152
:1013C0001124680F711D8B01020F111D1092AB03C8
:1013D000EB0115C085E06D2F0E94BB0286E06C2FEB
:1013E0000E94BB028091AB03F701E80FF11D608101
:1013F0008F5F8093AB0387E00E94BB022196C017EA
:10140000D10740F3DF91CF911F910F91FF90EF90A3
:1014100008956091030181E04DE051E025E00E94D4
:10142000D6090895DF93CF9300D000D0CDB7DEB7B3
:10143000F894309153027894832F6AE00E94DC196B
:10144000282F0E94DC19482F822F0E94DC19292F97
:10145000832F0E94DC19992319F48AE08C8301C040
:101460009C83222319F48AE08A8301C02A8349835A
:1014700085E48B8383E061E0AE014F5F5F4F24E042
:101480000E94D6090F900F900F900F90CF91DF918F
:101490000895DF93CF9300D000D0CDB7DEB780E2C0
:1014A00089839BE09A8381E38B839C8381E061E065
:1014B000AE014F5F5F4F21E00E94D60980919901F4
:1014C000813079F462E0AE014E5F5F4F21E00E940F
:1014D000D60981E063E0AE014D5F5F4F22E00E94DC
:1014E000D6090F900F900F900F90CF91DF91089534
:1014F000DF93CF9300D000D00F92CDB7DEB7DE01DF
:101500001196E1E4F1E085E001900D928150E1F760
:10151000609104018CE0AE014F5F5F4F25E00E94B7
:10152000D6090F900F900F900F900F90CF91DF91F1
:10153000089580E06CE40E94BB020895809121032D
:1015400090912203843B910554F08091A30390E095
:1015500020911F03309120038217930744F080915C
:10156000C901882371F481E08093C90108958091B5
:10157000C901181624F480E06CE40E94BB021092AA
:10158000C901089580E062E40E94BB0208958F9231
:101590009F92AF92BF92CF92DF92EF92FF920F9302
:1015A0001F93DF93CF93CDB7DEB72F970FB6F89485
:1015B000DEBF0FBECDBFFE013B9685E0DF011D9271
:1015C0008A95E9F780914F02909150026EE170E0A8
:1015D0000E94FC19CB01019797FF02C080E090E0C8
:1015E0008E010F5F1F4FB8014AE050E00E94AB1917
:1015F000F80101900020E9F73197FE2EF01A80E003
:10160000CF2CDD24C7FCD094F6E08F2E912C8C0ECD
:101610009D1E58010BC0F501E00FF11F80810E9453
:10162000F505080D191DF80180838E2D082F10E097
:10163000E82EE3940C151D0574F38093AB0385E14C
:1016400069E0AE01455F5F4F25E00E94D60989E160
:101650008F1969E0A4012F2D0E94D6092F960FB68D
:10166000F894DEBF0FBECDBFCF91DF911F910F91D8
:10167000FF90EF90DF90CF90BF90AF909F908F90B2
:1016800008958F929F92AF92BF92CF92DF92EF9286
:10169000FF920F931F93DF93CF93CDB7DEB72E97B3
:1016A0000FB6F894DEBF0FBECDBF19821A821B821F
:1016B0001C828091AE019091AF018E010B5F1F4F94
:1016C000B8014AE050E00E94AB19F80101900020F7
:1016D000E9F73197FE2EF01A80E0CF2CDD24C7FC0D
:1016E000D094AAE08A2E912C8C0E9D1E58010BC01E
:1016F000F501E00FF11F80810E94F505080D191D0D
:10170000F80180838E2D082F10E0E82EE3940C154D
:101710001D0574F38093AB0385E166E0AE014F5F76
:101720005F4F24E00E94D60989E18F1966E0A40189
:101730002F2D0E94D6098091AE019091AF0118160D
:10174000190664F485E060E00E94BB0286E062EC6A
:101750000E94BB0287E06CE80E94BB028091AE0150
:101760009091AF0197FF0CC085E060E00E94BB0242
:1017700086E062EC0E94BB0287E06DE80E94BB023B
:101780008091AE019091AF01892B61F485E060E01A
:101790000E94BB0286E062EC0E94BB0287E060E030
:1017A0000E94BB022E960FB6F894DEBF0FBECDBFCF
:1017B000CF91DF911F910F91FF90EF90DF90CF902D
:1017C000BF90AF909F908F9008958F929F92AF920D
:1017D000BF92CF92DF92EF92FF920F931F93DF930E
:1017E000CF93CDB7DEB72B970FB6F894DEBF0FBE01
:1017F000CDBFDE011196EEE3F1E083E001900D92A2
:101800008150E1F78E010C5F1F4F80911D03909175
:101810001E03B8014AE050E00E94AB19F8010190A4
:101820000020E9F73197FE2EF01A80E0CF2CDD245E
:10183000C7FCD094B8E08B2E912C8C0E9D1E5801C5
:101840000BC0F501E00FF11F80810E94F505080D26
:10185000191DF80180838E2D082F10E0E82EE394E7
:101860000C151D0574F38093AB038DE06EE0AE01A3
:101870004F5F5F4F23E00E94D60980E18F196EE031
:10188000A4012F2D0E94D6092B960FB6F894DEBF27
:101890000FBECDBFCF91DF911F910F91FF90EF90C1
:1018A000DF90CF90BF90AF909F908F9008958F92D0
:1018B0009F92AF92BF92DF92EF92FF920F931F938E
:1018C000DF93CF93CDB7DEB728970FB6F894DEBF7E
:1018D0000FBECDBF19828AE08A838091A0019091CA
:1018E000A1018E010D5F1F4FB8014AE050E00E9438
:1018F000AB19F80101900020E9F73197E01B80E077
:10190000EE2EFF24E7FCF094480106E0A02EB12C57
:10191000AC0EBD1E0BC0F401E00FF11F80810E94D0
:10192000F5050A0D1B1DF80180838D2D082F10E091
:10193000D82ED3940E151F0574F38093AB038091BA
:10194000A0019091A1018E010A5F1F4F0A977CF4BC
:101950006091030181E0AE014F5F5F4F21E00E9483
:10196000D6096091030182E0A80121E005C06091E1
:10197000030181E0A80122E00E94D6098091A20122
:101980009091A3018E010D5F1F4FB8014AE050E016
:101990000E94AB19F80101900020E9F73197E01B94
:1019A00080E0EE2EFF24E7FCF094480116E0A12E23
:1019B000B12CAC0EBD1E0BC0F401E00FF11F8081F5
:1019C0000E94F5050A0D1B1DF80180838D2D082F3F
:1019D00010E0D82ED3940E151F0574F38093AB033B
:1019E0008091A2019091A3018E010A5F1F4F0A9777
:1019F0007CF46091030184E0AE014E5F5F4F21E013
:101A00000E94D6096091030185E0A80121E005C08C
:101A10006091030184E0A80122E00E94D609289683
:101A20000FB6F894DEBF0FBECDBFCF91DF911F91EF
:101A30000F91FF90EF90DF90BF90AF909F908F90AD
:101A400008950F931F93DF93CF93CDB7DEB72A97F7
:101A50000FB6F894DEBF0FBECDBF8E010F5F1F4FD4
:101A6000B8014AE050E00E94AB19F8010190002053
:101A7000E9F73197E01B20E0FF27E7FDF095322FD3
:101A80003F5F822F90E08E179F0714F4232FF7CF2C
:101A90002093AB032A960FB6F894DEBF0FBECDBFDE
:101AA000CF91DF911F910F910895AF92BF92CF9286
:101AB000DF92EF92FF920F931F93DF93CF93CDB7F7
:101AC000DEB76E970FB6F894DEBF0FBECDBFB82E4F
:101AD000A62ED42EA42FB52FFD0101900020E9F7EA
:101AE0003197CE2EC41A7E010894E11CF11C242FDC
:101AF000352FC9018C0108C0F80181918F010E9426
:101B0000F505F70181937F01802F8D198C15A0F3C6
:101B10008B2D6A2DAE014F5F5F4F2C2D0E94D60991
:101B20006E960FB6F894DEBF0FBECDBFCF91DF919A
:101B30001F910F91FF90EF90DF90CF90BF90AF90EB
:101B4000089580919801813071F46091060120918F
:101B5000DF013091E001369527958EE0821B41EE42
:101B600051E00E94550D0895EF92FF920F931F933D
:101B7000DF93CF93CDB7DEB764970FB6F894DEBF8F
:101B80000FBECDBFF82EE62ECA018E010F5F1F4F8C
:101B9000B8014AE050E00E94AB198F2D6E2DA801CC
:101BA0000E94550D64960FB6F894DEBF0FBECDBFF0
:101BB000CF91DF911F910F91FF90EF900895EF92D9
:101BC000FF920F931F93DF93CF93CDB7DEB72A9782
:101BD0000FB6F894DEBF0FBECDBF20915C03822FFD
:101BE0006AE00E94DC19382F822F0E94DC1985E4FC
:101BF0008F8380915D03882309F48AE08887992385
:101C000019F48AE08E8301C09E833D8319821A8273
:101C10001B821C828E010B5F1F4F83E062E0A801D4
:101C200024E00E94D6098091600390916103B8017D
:101C30004AE050E00E94AB19F80101900020E9F75A
:101C40007F010894E108F108E01AF10A83E063E0FB
:101C5000AE014F5F5F4F24E00E94D60987E08E19E6
:101C600063E0A8010E94550D2A960FB6F894DEBFD6
:101C70000FBECDBFCF91DF911F910F91FF90EF90DD
:101C80000895BF92CF92DF92EF92FF920F931F932E
:101C9000DF93CF93CDB7DEB764970FB6F894DEBF6E
:101CA0000FBECDBFC82EB62EFA017E010894E11CEE
:101CB000F11C04C0AE0DBF1D9C9331968E2F841B6A
:101CC0009491A82FB0E09923A9F7AE0DBF1D1C92E7
:101CD000F70101900020E9F73197DE2EDE18870129
:101CE00007C0F80180810E94F505F80181938F01FA
:101CF000802F8E198D15A8F38C2D6B2DAE014F5FA3
:101D00005F4F2D2D0E94D60964960FB6F894DEBF62
:101D10000FBECDBFCF91DF911F910F91FF90EF903C
:101D2000DF90CF90BF9008951F93CF93DF93EC0186
:101D3000A3E0B0E047C0FD01EB58FD4F8081FD01FD
:101D4000EA58FD4F2081422F50E04D535040FD0195
:101D5000E958FD4F7081FD01E858FD4F10819A014F
:101D6000F4E035952795FA95E1F790E0CD97880F47
:101D7000991F880F991F282B392B2883613029F14F
:101D8000E72FF0E0FD9734E0440F551F3A95E1F757
:101D90005070CF019595879595958795482B592B30
:101DA0004983623091F01496635086E0EE0FFF1F76
:101DB0008A95E1F7F070812F90E0CD97E82BF92B11
:101DC000EA832396662309F0B6CFDF91CF911F9166
:101DD0000895809177028635B1F48091760281561C
:101DE0008093BA018091BA01843018F084E0809326
:101DF000BA018DE493E06AE043E02AE00E94940E89
:101E000081E08093BB011092950108951F9310917A
:101E1000BA01123009F486C0143009F4DBC0113065
:101E200009F09BC180917702813581F489E893E0C4
:101E30006BE143E02DE20E94940E8091890390E0D3
:101E40009093BD018093BC011093C00180917702F3
:101E5000843409F082C18BE093E061E443E021E443
:101E60000E94940E8091210390912203843B91055E
:101E700054F480919A01813031F410929A01F894CF
:101E80000E94C11078948091210390912203843B99
:101E900091057CF080919A01882359F481E0809328
:101EA0009A01F89480919701882311F40E94B1104F
:101EB000789480910D0390910E0366E170E00E948A
:101EC000FC196E5F7F4F70934E0260934D028091BC
:101ED0000F039091100366E170E00E94FC196A5FA5
:101EE0007F4F70934C0260934B0280911703909147
:101EF00018039093500280934F0280911F038093A8
:101F00005302809132029091330290935202809357
:101F1000510280911D0390911E039093560280936D
:101F200055021BC1809177028F34A9F0813509F0E9
:101F300014C189E893E06CE143E02DE20E94940E25
:101F40008091890390E09093BD018093BC0181E072
:101F50008093C00102C185EF91E060E543E02DE28E
:101F60000E94940E80913D02992787FD90950296DC
:101F700090934E0280934D0280913E02992787FDF7
:101F80009095069690934C0280934B02809130027C
:101F9000909131029093500280934F0280913602CB
:101FA00080935302809132029091330290935202B7
:101FB0008093510280913B0290913C029093560293
:101FC0008093550280912F028093570281E0809385
:101FD000BF01C3C080917702843409F05AC08BE0FE
:101FE00093E061E443E021E40E94940E8091210398
:101FF00090912203843B910554F480919A018130A1
:1020000031F410929A01F8940E94C1107894809152
:10201000210390912203843B91057CF080919A01E9
:10202000882359F481E080939A01F8948091970174
:10203000882311F40E94B110789480910D0390913F
:102040000E0366E170E00E94FC196E5F7F4F709393
:102050004E0260934D0280910F039091100366E150
:1020600070E00E94FC196A5F7F4F70934C0260938E
:102070004B02809117039091180390935002809324
:102080004F0280911D0390911E03909356028093FE
:102090005502809177028C3481F481E090E0909336
:1020A000BD018093BC0181E08093C0018BE893E087
:1020B00069E143E02DE20E94940E809177028D3415
:1020C00081F482E090E09093BD018093BC0181E0B7
:1020D0008093C0018BE893E069E143E02DE20E9428
:1020E000940E809177028E3481F483E090E0909397
:1020F000BD018093BC0181E08093C0018BE893E037
:1021000069E143E02DE20E94940E809177028F34C2
:1021100081F484E090E09093BD018093BC0181E064
:102120008093C0018BE893E069E143E02DE20E94D7
:10213000940E80917702803581F485E090E0909351
:10214000BD018093BC0181E08093C0018BE893E0E6
:1021500069E143E02DE20E94940E109295011F91D7
:10216000089582E289B910BC80B91CBE909A28E912
:102170002AB996E890BD82EC8BB921B99CBF82B98F
:10218000089582E289B910BC80B91CBE88E98AB979
:1021900026E820BD92EC9BB980E981B92CBF92B9A9
:1021A0000895DF93CF93CDB7DEB72C970FB6F89491
:1021B000DEBF0FBECDBF83E2898383E68A8385E7D6
:1021C0008B838DE38C838D838E838F83DE011196C9
:1021D000FD0120E030E0AE01485F5F4F8191280FA4
:1021E000311DE417F507D1F7C9019F7046E09595B9
:1021F00087954A95E1F7835C88872F733070822F2B
:10220000835C89878DE08A879E01255F3F4F8C9193
:10221000159BFECF83B91196A217B307C1F72C9671
:102220000FB6F894DEBF0FBECDBFCF91DF910895FA
:10223000DF93CF93CDB7DEB72C970FB6F894DEBF00
:102240000FBECDBF8BE189838A8385E58B838AEAC4
:102250008C831D82FE0131969E012A5F3F4F808153
:10226000159BFECF83B93196E217F307C1F72C9681
:102270000FB6F894DEBF0FBECDBFCF91DF910895AA
:10228000DF93CF93CDB7DEB72A970FB6F894DEBFB2
:102290000FBECDBF93E299838A836B83842F86958B
:1022A0008695835C8C8350E04370507064E0440FEB
:1022B000551F6A95E1F7435C4D838DE38E838F83D1
:1022C000DE011196FD0120E030E0AE01485F5F4F76
:1022D0008191280F311DE417F507D1F7C9019F70CF
:1022E00056E0959587955A95E1F7835C88872F731B
:1022F0003070822F835C89878DE08A879E01255FFD
:102300003F4F8C91159BFECF83B91196A217B3074F
:10231000C1F72A960FB6F894DEBF0FBECDBFCF919E
:10232000DF9108955D9BFECF8DE68CB95D9BFECF5E
:102330008FE68CB95D9BFECF89E68CB95D9BFECFA5
:102340008EE68CB95D9BFECF8DE08CB95D9BFECF98
:102350008EE38CB90895982F9F7082958F708A3084
:1023600010F4805D01C0895C5D9BFECF8CB99A3012
:1023700018F4892F805D02C0892F895C5D9BFECF98
:102380008CB908958A3010F4805D01C0895C5D9B32
:10239000FECF8CB90895159BFECF83B908955D9B40
:1023A000FECF8CB90895662359F020E0FC01E20FBE
:1023B000F11DE0815D9BFECFECB92F5F6217B0F796
:1023C00008955D9BFECF8EE38CB908951F920F9206
:1023D0000FB60F9211242F933F938F939F93AF9338
:1023E000BF93EF93FF932CB12093AC0385B398E098
:1023F000892785BB5D9BFECF2CB92D3059F080918C
:102400008803E82FF0E0EE59FC4F20838F5F809324
:10241000880359C0E0918803F0E0EE59FC4F208317
:102420001092B7011092B8011092B90130E020E08B
:1024300090E03FC02130B9F0213018F02230C1F5D2
:1024400024C0A32FB0E0AE59BC4F8C91803211F460
:1024500021E023C0E92FF0E08C91E058FC4F80830D
:102460009093B70124C0A32FB0E0AE59BC4F8C911C
:10247000803211F422E011C0E92FF0E08C91E8598C
:10248000FD4F80839093B80112C0A32FB0E0AE59E6
:10249000BC4F8C91803219F423E090E009C0E92F01
:1024A000F0E08C91E75AFD4F80839093B9019F5FD4
:1024B0003F5F80918803831708F0BCCF81E0809351
:1024C000B60110928803FF91EF91BF91AF919F9158
:1024D0008F913F912F910F900FBE0F901F901895E5
:1024E0001F920F920FB60F9211248F939F93EF9329
:1024F000FF9393B19093AD039D3081F48091CA0115
:10250000813061F4AB981092CA0180939501E091FB
:102510005803F0E0EB58FD4F90832DC08091CA0125
:10252000882319F0813039F514C0933241F4809139
:102530009501882321F481E08093CA01AB9A10921F
:10254000580380915803E82FF0E0EB58FD4F90833B
:102550000CC0E0915803F0E0EB58FD4F9083809160
:102560005803853930F4809158038F5F8093580366
:1025700002C01092CA01FF91EF919F918F910F902D
:102580000FBE0F901F90189585B392E0892785BBE9
:10259000089590919D01913019F485B3892785BBE9
:1025A00008951F920F920FB60F9211242F933F930D
:1025B0005F936F937F938F939F93AF93BF9380911C
:1025C000CC019091CD01892B81F484B595B5909380
:1025D000D3018093D2018EB58F7B8EBD81E090E0D8
:1025E0009093CD018093CC013AC084B595B590937A
:1025F000D1018093D0012EB520642EBD2091D2014F
:102600003091D3011092CD011092CC01821B930B1B
:10261000865698406CE271E00E94E8197093CF01F1
:102620006093CE016730710534F086E090E09093BE
:10263000CF018093CE012091CE013091CF018091C6
:102640000201992787FD90952817390741F0263018
:1026500031052CF42093020181E08093A401BF9105
:10266000AF919F918F917F916F915F913F912F914A
:102670000F900FBE0F901F90189580914F02909170
:1026800050029093A7018093A6018091A60190919A
:10269000A7012091A8013091A901821B930B90936F
:1026A000AB018093AA018091A6019091A70190931C
:1026B000A9018093A8014091B2015091B30180918A
:1026C000AA019091AB01E3E0880F991FEA95E1F729
:1026D0009A0173E0220F331F7A95E1F7241B350B23
:1026E000820F931F68E070E00E94FC197093B301A1
:1026F0006093B2012091B4013091B5014091B201D3
:102700005091B301C90163E0880F991F6A95E1F701
:10271000821B930B840F951F68E070E00E94FC19E8
:102720007093B5016093B4018091B4019091B501AB
:102730009093AF018093AE010E94410B08958AE10E
:1027400061E04EE451E022E00E94D6090895DF9353
:10275000CF9300D00F92CDB7DEB7DE011196E0E542
:10276000F1E083E001900D928150E1F76091040166
:102770006F5F8EE0AE014F5F5F4F23E00E94D6098E
:10278000609104016F5F4091290250912A028EE00E
:102790000E94B40D0F900F900F90CF91DF9108958C
:1027A000DF93CF9300D00F92CDB7DEB7DE01119645
:1027B000E3E5F1E083E001900D928150E1F7609153
:1027C00004018EE0AE014F5F5F4F23E00E94D60907
:1027D0006091040140912B0250912C028EE00E94E6
:1027E000B40D0F900F900F90CF91DF9108958F92BD
:1027F0009F92BF92CF92DF92EF92FF920F931F931F
:10280000DF93CF93CDB7DEB72B970FB6F894DEBF2B
:102810000FBECDBFDE011196E6E5F1E083E0019049
:102820000D928150E1F7809157028E010C5F1F4F8E
:1028300090E0B8014AE050E00E94AB19F801019025
:102840000020E9F73197BE2EB01AEE24FF24CB2CDE
:10285000DD24C7FCD09488E0882E912C8C0E9D1E20
:102860000DC0F801EE0DFF1D80810E94F505F401F9
:10287000EE0DFF1D80830894E11CF11CEC14FD0497
:1028800084F388E161E0AE014F5F5F4F23E00E9477
:10289000D6098BE18B1961E0A4012B2D0E94D6098A
:1028A0002B960FB6F894DEBF0FBECDBFCF91DF9150
:1028B0001F910F91FF90EF90DF90CF90BF909F906E
:1028C0008F90089583E66FE644E60E944011F894E5
:1028D00028E088E190E00FB6F894A89581BD0FBE7E
:1028E00021BDFFCF1F939D998AC18091D4018F5F35
:1028F0008093D40111E01093D6018091D4018530EA
:1029000009F081C18091D801882309F08CC010930F
:10291000D8011092D90184E064E00E94BB0283E0F8
:1029200061E041EE51E00E94550D83E063E040E13B
:1029300052E00E94410E84E068E00E94BB0283E006
:1029400065E049E152E00E94410E80910001813032
:1029500029F484E165E045E452E004C084E165E0E7
:1029600048E452E00E94410E84E060E00E94BB0215
:1029700083E066E04DE152E00E94410E80919701B4
:10298000813029F484E166E045E452E004C084E14A
:1029900066E048E452E00E94410E83E067E043E2D3
:1029A00052E00E94410E80919801813029F484E127
:1029B00067E045E452E004C084E167E048E452E0A7
:1029C0000E94410E83E068E04BE252E00E94410E1B
:1029D0008091A501813029F484E168E045E452E06A
:1029E00004C084E168E048E452E00E94410E83E0C4
:1029F00069E046E352E00E94410E809199018130E6
:102A000029F484E169E045E452E004C084E169E02E
:102A100048E452E00E94410E83E06BE040E452E063
:102A20000E94410EEEC08091D901882349F584E0CF
:102A300068E00E94BB0280910001882339F4109362
:102A4000000184E165E045E452E006C01092000117
:102A500084E165E048E452E00E94410E20910001CB
:102A6000E199FECF81E090E09FBB8EBB2DBB0FB6FE
:102A7000F894E29AE19A0FBE84E060E00E94BB0203
:102A80001091D901113049F584E068E00E94BB0241
:102A900080919701882339F41093970184E166E0CF
:102AA00045E452E006C01092970184E166E048E4F4
:102AB00052E00E94410E20919701E199FECF80E003
:102AC00090E09FBB8EBB2DBB0FB6F894E29AE19AC3
:102AD0000FBE84E060E00E94BB028091D901823089
:102AE00051F584E068E00E94BB0280919801882340
:102AF00041F481E08093980184E167E045E452E08D
:102B000006C01092980184E167E048E452E00E9418
:102B1000410E20919801E199FECF82E090E09FBBA9
:102B20008EBB2DBB0FB6F894E29AE19A0FBE84E0FB
:102B300060E00E94BB028091D901833051F584E0AE
:102B400068E00E94BB028091A501882341F481E0E6
:102B50008093A50184E168E045E452E006C010924C
:102B6000A50184E168E048E452E00E94410E209112
:102B7000A501E199FECF87E190E09FBB8EBB2DBB05
:102B80000FB6F894E29AE19A0FBE84E060E00E94EA
:102B9000BB028091D901843049F568E00E94BB02F4
:102BA00080919901882341F481E08093990184E127
:102BB00069E045E452E006C01092990184E169E0C1
:102BC00048E452E00E94410E20919901E199FECF24
:102BD0008BE190E09FBB8EBB2DBB0FB6F894E29AC1
:102BE000E19A0FBE84E060E00E94BB028091D901AF
:102BF000853049F41092D8010E94621404C01092EA
:102C0000D4011092D6019C9913C19091D8019130B2
:102C100009F014C19093D7018091D5018F5F809303
:102C2000D5012091D501253009F008C11092D501B8
:102C30008091D901823009F469C0833030F488234F
:102C400071F0813009F0FAC035C0843009F4AAC0AF
:102C5000843008F486C0853009F0F0C0C3C090937A
:102C6000D90183E065E049E152E00E94410E809184
:102C70000001813029F484E165E045E452E004C0BC
:102C800084E165E048E452E00E94410E84E068E09F
:102C90000E94BB0283E066E04DE152E00E94410EDB
:102CA00080919701813019F484E166E0B3C084E13A
:102CB00066E0B5C082E08093D90183E066E04DE133
:102CC00052E00E94410E80919701813029F484E105
:102CD00066E045E452E004C084E166E048E452E086
:102CE0000E94410E84E068E00E94BB0283E067E03E
:102CF00043E252E00E94410E80919801813019F424
:102D000084E167E087C084E167E089C083E0809365
:102D1000D90167E043E252E00E94410E80919801A0
:102D2000813029F484E167E045E452E004C084E1A5
:102D300067E048E452E00E94410E84E068E00E94AF
:102D4000BB0283E068E04BE252E00E94410E8091BA
:102D5000A501813019F484E168E05CC084E168E099
:102D60005EC084E08093D90183E068E04BE252E0EA
:102D70000E94410E8091A501813029F484E168E030
:102D800045E452E004C084E168E048E452E00E9477
:102D9000410E84E068E00E94BB0283E069E046E304
:102DA00052E03FC02093D90183E069E046E352E05E
:102DB0000E94410E80919901813029F484E169E0FB
:102DC00045E452E004C084E169E048E452E00E9436
:102DD000410E84E068E00E94BB0283E06BE040E4C7
:102DE00052E01FC01092D90183E06BE040E452E052
:102DF0000E94410E84E068E00E94BB0283E065E02F
:102E000049E152E00E94410E80910001813029F495
:102E100084E165E045E452E004C084E165E048E413
:102E200052E00E94410E84E060E00E94BB0206C0B6
:102E30001092D5018091D6018091D7011F910895FC
:102E4000813061F4E199FECF80E090E09FBB8EBBC2
:102E50006DBB0FB6F894E29AE19A0FBE0895DF9326
:102E6000CF93CDB7DEB764970FB6F894DEBF0FBE31
:102E7000CDBF20E0DE011196E199FECFE22FF0E018
:102E8000CF018D5F9F4F9FBB8EBBE09A8DB3EA0F42
:102E9000FB1F8083882311F02F5FEECFFD0101908F
:102EA0000020E9F79F01215030402A1B3B0B309353
:102EB000E0012093DF0190E0AE014F5F5F4F09C05A
:102EC000FD01EF51FE4FA40FB51F8C91808311823D
:102ED0009F5FA92FB0E0A217B30790F364960FB6D7
:102EE000F894DEBF0FBECDBFCF91DF910895DF9381
:102EF000CF93CDB7DEB760970FB6F894DEBF0FBEA5
:102F0000CDBF8091550290915602909374028093A8
:102F1000730280917302909174026FE070E00E94DE
:102F2000E819DE011596AD016A1B9E01205F3F4F37
:102F3000E62FEA0FF0E0E55BFD4FE491ED93A21779
:102F4000B307B1F76091070119821A821B821C82B4
:102F500089E02BE00E94D609609108018EE0AE0165
:102F60004F5F5F4F24E00E94D609609108014091B5
:102F70007302509174028FE00E94B40D60960FB6F8
:102F8000F894DEBF0FBECDBFCF91DF910895DF93E0
:102F9000CF93CDB7DEB7E2970FB6F894DEBF0FBE82
:102FA000CDBFDE011796E9E5F1E087E001900D92D3
:102FB0008150E1F7DE011E96E0E6F1E089E0019044
:102FC0000D928150E1F7DE015796E9E6F1E08EE0DF
:102FD00001900D928150E1F7DE011196E7E7F1E0F3
:102FE00086E001900D928150E1F7DE019596EDE7C4
:102FF000F1E08EE001900D928150E1F75091800355
:1030000060918103409182038091830320E030E04E
:10301000803711F421E030E080E090E04C3611F48C
:1030200081E090E02823392380E0583609F481E0DC
:1030300090E0653609F491E0892390E02823392354
:10304000232B79F0CE01079666E00E94D311CE01C2
:103050000E9668E00E94D311CE0147966DE00E9463
:10306000D31150918003609181034091820380913C
:10307000830320E030E0873711F421E030E080E086
:1030800090E04F3611F481E090E02823392380E06E
:10309000533709F481E090E0683609F491E0892320
:1030A00090E028233923232B19F180916802909115
:1030B0006902893481F4943471F4CE01019665E09B
:1030C0000E94D31181EE91E06091DF010E94D31143
:1030D0008DE00E94CF11809168029091690286373D
:1030E00039F4953629F4CE0185966CE00E94D3110F
:1030F00080918003209181034091820390E0833787
:1031000009F491E080E0253609F481E09823892FC5
:1031100090E020E030E0443711F421E030E08223F9
:103120009323892B09F442C080916802909169022F
:10313000893409F03BC0943409F038C020E01AC04B
:10314000FD01E75AFD4FE081E199FECF822F90E02B
:103150008D5F9F4F9FBB8EBBEDBB0FB6F894E29A7D
:10316000E19A0FBEFD01E75AFD4F8081AF51BE4F7E
:103170008C932F5F8091B901A22FB0E0281700F344
:10318000E199FECFCD018D5F9F4F9FBB8EBB1DBAD6
:103190000FB6F894E29AE19A0FBEE22FF0E0EF51F9
:1031A000FE4F1082B093E001A093DF0150918003A5
:1031B00060918103409182038091830320E030E09D
:1031C000853611F421E030E080E090E0433711F4DF
:1031D00081E090E02823392380E0523709F481E030
:1031E00090E0653609F491E0892390E028233923A3
:1031F000232B11F00E9462140E94E111E2960FB697
:10320000F894DEBF0FBECDBFCF91DF9108951F921E
:103210000F920FB60F9211242F933F938F939F938A
:10322000EF93FF938091DB01882381F08091DB0194
:1032300090E00197E0918D01F0918E01E80FF91F68
:103240008FB1808381E08093DC0103C08FB18093D4
:10325000B3032091DB0180918B0130E0992787FD3A
:103260009095821793075CF084E080938C0181E055
:103270008093DC018091DB018093B20308C0929AB5
:103280001092DA0181E08093DD011092DE018091DD
:10329000DB018F5F8093DB01FF91EF919F918F9115
:1032A0003F912F910F900FBE0F901F90189582EDB8
:1032B0008DB90895813029F4613011F49298089500
:1032C000929A0895982F8091DA018823C9F4913059
:1032D00009F492989093DA0181E08093DE019130B5
:1032E00069F486E080938B011092DB018AE0809381
:1032F0008C019093DC018AEA8093B20380E0089508
:103300008091DC01813071F480918C018150809337
:103310008C018F5F39F48091B2038FB91092DC0178
:1033200081E0089581E00895CF93DF93C0E0D0E07D
:10333000E0918D01F0918E01EC0FFD1F80810E94C4
:10334000AB112196C730D10599F78DE00E94CF11BE
:10335000DF91CF910895FB019F01E8944230C4F0C2
:103360004532B4F44A3029F497FB1EF490958195C8
:103370009F4F642F77270E94E819805D8A330CF0F5
:10338000895D8193CB010097A1F716F45DE251931B
:103390001082C9010C94CC19DC01FC01672F7191DA
:1033A0007723E1F7329704C07C916D93708362912B
:1033B000AE17BF07C8F30895991B79E004C0991FA1
:1033C000961708F0961B881F7A95C9F7809508957F
:1033D000AA1BBB1B51E107C0AA1FBB1FA617B7073B
:1033E00010F0A61BB70B881F991F5A95A9F7809557
:1033F0009095BC01CD01089597FB092E07260AD0B0
:1034000077FD04D0E5DF06D000201AF470956195B1
:103410007F4F0895F6F7909581959F4F0895F89402
:02342000FFCFDC
:103422000101030E0786010E0C5C00000A00004435
:103432000000230023005464665363655262005106
:10344200610050600050600051610052620053639D
:10345200655464666768696A6B6B6A6968670000CD
:103462000053536353530B03F50189030D0A0A1DDD
:1034720000000000000000000068656C70200D0074
:1034820073686F772049440D0073686F7720766503
:103492007273696F6E0D004944203D2000302E3951
:1034A2002E312E382E626574610D0009075B030010
:00000001FF
